:100000007F28A0008417800484138E010C1C8E00AE
:10001000102003197A28102003197A2810207A2832
:1000200020088E0601308C008D01000820050E0688
:10003000031D08008C0A03198D0F152808008F0076
:10004000220884002009462084138F0803197A2887
:10005000F03091000E0880389000F03091030319C1
:10006000910003198F0303197A28362849200301C8
:100070000C1820088E1F20088E0803190301900F0A
:10008000432880062A28442800002D28841780054C
:100090007A280D080C0403198C0A80300C1A8D067E
:1000A0000C198D068C188D060D0D8C0D8D0D7A2872
:1000B0008F018E00FF308E07031C8F07031C7A28E8
:1000C00003308D00DF3066205A288D01E83E8C0019
:1000D0008D09FC30031C6F288C0703186C288C07D3
:1000E00064008D0F6C280C1875288C1C7928000072
:1000F0007928080083130313831264000800831611
:10010000033085000830860083128610831686101F
:10011000831206108316061006308312A2001030D8
:10012000A00064308E000A301F2032308E0005306F
:100130001F2046308E000A301F2032308E000230E1
:100140001F2001308C0005308400013001200C0894
:10015000A40001308C0005308400023001200C081E
:10016000A5006400B5302502031CCA280630A20091
:100170001030A00064308E000A301F2032308E0014
:1001800005301F200614831606108312861083166E
:10019000861083126400783025020318E7280630A1
:1001A000A2001030A00032308E0005301F206430D5
:1001B0008E000A301F201E308E0014301F200610C3
:1001C0008316061083128614831686108312640029
:1001D00078302402031804290630A2001030A00051
:1001E00073308E000A301F2050308E0005301F20E3
:1001F00032308E0014301F2006148316061083122E
:1002000086148316861083126400B5302402031C02
:1002100036290630A2001030A00032308E00143093
:100220001F2050308E0005301F2073308E000A30A2
:100230001F200130A600640008302602031836296A
:1002400006148316061083128614831686106430F3
:100250008312582006108316061083128610831608
:100260008610643083125820A60F1B29A128630032
:0202700037292C
:02400E00F53F7C
:00000001FF
